******************************************************************************
               TMS320C6x Linker PC v7.4.2                      
******************************************************************************
>> Linked Fri Jan 03 14:04:31 2014

OUTPUT FILE NAME:   <Robust.out>
ENTRY POINT SYMBOL: "_c_int00"  address: 0c0182c0


MEMORY CONFIGURATION

         name            origin    length      used     unused   attr    fill
----------------------  --------  ---------  --------  --------  ----  --------
  VECTORS               00800000   00000200  00000200  00000000  RWIX
  LL2_CODE              00800200   0001fe00  000005c0  0001f840  RWIX
  LL2_DATA              00820000   00020000  0001a33c  00005cc4  RWIX
  SL2_CODE              0c000000   00080000  00018a00  00067600  RWIX
  SL2_DATA              0c080000   00040000  00036d5c  000092a4  RWIX
  SL2_REMAP             18000000   00040000  00000000  00040000  RWIX
  DDR3_CODE             80000000   01000000  00000000  01000000  RWIX
  DDR3_DATA             81000000   05000000  00028000  04fd8000  RWIX
  DDR3_Profile_DATA     86000000   02000000  00000000  02000000  RWIX
  DDR3_ECC_DATA         88000000   01000000  00000000  01000000  RWIX


SEGMENT ALLOCATION MAP

run origin  load origin   length   init length attrs members
----------  ----------- ---------- ----------- ----- -------
00800000    00800000    000007c0   000007c0    r-x
  00800000    00800000    00000200   00000200    r-x vecs
  00800200    00800200    00000480   00000480    r-x .text:Core_MPAX
  00800680    00800680    00000140   00000140    r-x ll2EDCCode
00820000    00820000    00018000   00000000    rw-
  00820000    00820000    00010000   00000000    rw- ll2MPData
  00830000    00830000    00008000   00000000    rw- .sysmem
00838000    00838000    00002194   00002074    rw-
  00838000    00838000    00001000   00001000    rw- .stack
  00839000    00839000    000009a0   000009a0    rw- .far
  008399a0    008399a0    000006d4   000006d4    rw- .fardata
  0083a074    0083a074    00000120   00000000    rw- .cio
0083a194    0083a194    00000108   000000f4    rw-
  0083a194    0083a194    000000f4   000000f4    rw- .neardata
  0083a288    0083a288    00000014   00000000    rw- .bss
0083a2c0    0083a2c0    000000a0   000000a0    rw-
  0083a2c0    0083a2c0    000000a0   000000a0    rw- ll2EDCData
0c000000    0c000000    00018a00   00018a00    r-x
  0c000000    0c000000    00018940   00018940    r-x .text
  0c018940    0c018940    000000c0   000000c0    r-x Sl2EDCCode
0c080000    0c080000    00027800   00000000    rw-
  0c080000    0c080000    00010000   00000000    rw- msmcSmsMPData_w
  0c090000    0c090000    00010000   00000000    rw- sl2MPData_w
  0c0a0000    0c0a0000    00007800   00000000    rw- PacketData.buffer_SL2
0c0a8000    0c0a8000    00008000   00000000    rw-
  0c0a8000    0c0a8000    00004000   00000000    rw- msmcSmsMPData_r
  0c0ac000    0c0ac000    00004000   00000000    rw- sl2MPData_r
0c0b0000    0c0b0000    00003480   00003480    r--
  0c0b0000    0c0b0000    00003480   00003480    r-- .const
0c0b3480    0c0b3480    00002880   00000000    rw-
  0c0b3480    0c0b3480    00002880   00000000    rw- QMSS_Data.Descriptor_SL2
0c0b6000    0c0b6000    00001000   00000000    rw-
  0c0b6000    0c0b6000    00001000   00000000    rw- Sl2EDCData
0c0b7000    0c0b7000    0000085c   0000085c    r--
  0c0b7000    0c0b7000    0000085c   0000085c    r-- .cinit
81000000    81000000    00028000   00000000    rw-
  81000000    81000000    00010000   00000000    rw- ddr3MPData_w
  81010000    81010000    00010000   00000000    rw- msmcSesMPData_w
  81020000    81020000    00004000   00000000    rw- ddr3MPData_r
  81024000    81024000    00004000   00000000    rw- msmcSesMPData_r


SECTION ALLOCATION MAP

 output                                  attributes/
section   page    origin      length       input sections
--------  ----  ----------  ----------   ----------------
vecs       0    00800000    00000200     
                  00800000    00000200     Robust_vectors.obj (vecs)

.text:Core_MPAX 
*          0    00800200    00000480     
                  00800200    00000440     KeyStone_common.obj (.text:Core_MPAX)
                  00800640    00000010     KeyStone_common.obj ($Tramp$S$$CSL_XMC_invalidatePrefetchBuffer)
                  00800650    00000010     KeyStone_common.obj ($Tramp$S$$CACHE_wbInvAllL2)
                  00800660    00000010     rts6600e_elf.lib : printf.obj ($Tramp$S$$printf)
                  00800670    00000010     --HOLE-- [fill = 0]

ll2EDCCode 
*          0    00800680    00000140     
                  00800680    00000100     Robust_LL2_EDC.obj (ll2EDCCode)
                  00800780    00000040     Robust_L1P_ED.obj (ll2EDCCode)

ll2MPData 
*          0    00820000    00010000     UNINITIALIZED
                  00820000    00010000     Robust_LL2_MP.obj (ll2MPData)

.sysmem    0    00830000    00008000     UNINITIALIZED
                  00830000    00000008     rts6600e_elf.lib : memory.obj (.sysmem)
                  00830008    00007ff8     --HOLE--

.stack     0    00838000    00001000     
                  00838000    00000008     rts6600e_elf.lib : boot.obj (.stack) [fill = bfbfbfbf]
                  00838008    00000ff8     --HOLE-- [fill = bfbfbfbf]

.far       0    00839000    000009a0     
                  00839000    00000400     Robust_LL2_MP.obj (.far) [fill = 0]
                  00839400    000002c0     Robust_System.obj (.far:Core_MPAX)
                  008396c0    00000140     rts6600e_elf.lib : defs.obj (.far) [fill = 0]
                  00839800    000000cc     Robust_SRIO_Init.obj (.far) [fill = 0]
                  008398cc    0000006c     KeyStone_common.obj (.far) [fill = 0]
                  00839938    00000020     Robust_DDR_XMC_MP.obj (.far:Core_MPAX)
                  00839958    00000020     Robust_SL2_XMC_MP.obj (.far:Core_MPAX)
                  00839978    00000010     KeyStone_DDR_Init.obj (.far:Core_MPAX)
                  00839988    00000010     KeyStone_common.obj (.far:Core_MPAX)
                  00839998    00000008     rts6600e_elf.lib : trgdrv.obj (.far) [fill = 0]

.fardata   0    008399a0    000006d4     
                  008399a0    000001e0     rts6600e_elf.lib : defs.obj (.fardata:_ftable)
                  00839b80    000000a0                      : lowlev.obj (.fardata:_stream)
                  00839c20    00000084     Robust_Peripherals_MPU.obj (.fardata:MPU2_cfg_table)
                  00839ca4    00000004     rts6600e_elf.lib : defs.obj (.fardata)
                  00839ca8    00000078                      : lowlev.obj (.fardata:_device)
                  00839d20    00000078     Robust_MNav_Init.obj (.fardata:freeHostQueueCfgTable)
                  00839d98    00000070     Robust_MNav_Init.obj (.fardata:flowCfgTable)
                  00839e08    00000048     KeyStone_SRIO_Init_drv.obj (.fardata:LSU_state_index_table)
                  00839e50    00000040     KeyStone_common.obj (.fardata:gstruMpuAddrRange)
                  00839e90    0000003c     Robust_Peripherals_MPU.obj (.fardata:MPU1_cfg_table)
                  00839ecc    00000004     --HOLE--
                  00839ed0    00000024     KeyStone_common.obj (.fardata:gpTimerRegs)
                  00839ef4    00000004     --HOLE--
                  00839ef8    00000024     KeyStone_common.obj (.fardata:internal_exception_str)
                  00839f1c    00000004     --HOLE--
                  00839f20    00000020     Robust_DDR_SES_MP.obj (.fardata:SES_MPAX_cfg_table)
                  00839f40    00000020     Robust_SL2_SMS_MP.obj (.fardata:SMS_MPAX_cfg_table)
                  00839f60    00000020     KeyStone_common.obj (.fardata:bus_err_stat_str)
                  00839f80    00000020     KeyStone_common.obj (.fardata:gCIC_EXC_EN_MASK)
                  00839fa0    00000020     KeyStone_common.obj (.fardata:gpMPU_regs)
                  00839fc0    00000018     KeyStone_common.obj (.fardata:Peri_MPU_err_type_str)
                  00839fd8    00000018     Robust_MNav_Init.obj (.fardata:descMemRegionsCfg)
                  00839ff0    00000014     Robust_SRIO_Init.obj (.fardata:path_str)
                  0083a004    00000004     --HOLE--
                  0083a008    00000010     Robust_MNav_Init.obj (.fardata:freeMonoQueueCfgTable)
                  0083a018    00000010     KeyStone_common.obj (.fardata:gpEDMA_TC_regs)
                  0083a028    0000000c     rts6600e_elf.lib : exit.obj (.fardata)
                  0083a034    0000000c                      : memory.obj (.fardata)
                  0083a040    00000008     KeyStone_common.obj (.fardata:Ns_str)
                  0083a048    00000008     KeyStone_Navigator_init_drv.obj (.fardata:gpQM_PDSP_Cmd)
                  0083a050    00000008     KeyStone_Navigator_init_drv.obj (.fardata:gpQM_PDSP_CtrlRegs)
                  0083a058    00000008     KeyStone_Navigator_init_drv.obj (.fardata:gpQM_PDSP_IRAM)
                  0083a060    00000008     rts6600e_elf.lib : _lock.obj (.fardata)
                  0083a068    00000006     Robust_SRIO_Init.obj (.fardata:dsp0_device_ID_routing_config)
                  0083a06e    00000002     --HOLE--
                  0083a070    00000004     KeyStone_common.obj (.fardata:gpEDMA_CC_regs)

.cio       0    0083a074    00000120     UNINITIALIZED
                  0083a074    00000120     rts6600e_elf.lib : trgmsg.obj (.cio)

.neardata 
*          0    0083a194    000000f4     
                  0083a194    00000098     KeyStone_common.obj (.neardata)
                  0083a22c    00000050     KeyStone_Navigator_init_drv.obj (.neardata)
                  0083a27c    00000004     KeyStone_SRIO_Init_drv.obj (.neardata)
                  0083a280    00000004     Robust_INTC.obj (.neardata)
                  0083a284    00000004     Robust_SRIO_Init.obj (.neardata)

.rodata    0    0083a288    00000000     UNINITIALIZED

.bss       0    0083a288    00000014     UNINITIALIZED
                  0083a288    00000010     Robust_MNav_Init.obj (.bss)
                  0083a298    00000004     KeyStone_SRIO_Init_drv.obj (.bss)

ll2EDCData 
*          0    0083a2c0    000000a0     
                  0083a2c0    00000080     Robust_LL2_EDC.obj (ll2EDCData)
                  0083a340    00000020     Robust_L1P_ED.obj (ll2EDCData) [fill = 0]

.text      0    0c000000    00018940     
                  0c000000    00005f00     KeyStone_common.obj (.text)
                  0c005f00    00002a20     KeyStone_DDR_Init.obj (.text)
                  0c008920    00002900     KeyStone_SRIO_Init_drv.obj (.text)
                  0c00b220    00001a80     KeyStone_Navigator_init_drv.obj (.text)
                  0c00cca0    00000a00     Keystone_Serdes_init.obj (.text)
                  0c00d6a0    000007c0     Robust_DDR_SES_MP.obj (.text)
                  0c00de60    00000780     Robust_SL2_SMS_MP.obj (.text)
                  0c00e5e0    00000700     Robust_LL2_EDC.obj (.text)
                  0c00ece0    000006a0     Robust_INTC.obj (.text:retain)
                  0c00f380    00000620     Robust_SL2_EDC.obj (.text)
                  0c00f9a0    00000600     KeyStone_common.obj (.text:retain)
                  0c00ffa0    000005e0     Robust_SRIO_Init.obj (.text)
                  0c010580    000005c0     Robust_System.obj (.text)
                  0c010b40    000005c0     rts6600e_elf.lib : divd.obj (.text:__c6xabi_divd)
                  0c011100    000005c0                      : _printfi.obj (.text:_getarg_diouxp)
                  0c0116c0    00000460                      : _printfi.obj (.text:_printfi)
                  0c011b20    00000460                      : _printfi.obj (.text:_setfield)
                  0c011f80    00000400     Robust_INTC.obj (.text)
                  0c012380    000003a0     rts6600e_elf.lib : fputs.obj (.text:fputs)
                  0c012720    00000320     Robust_LL2_MP.obj (.text)
                  0c012a40    00000320     rts6600e_elf.lib : _printfi.obj (.text:_pproc_fge)
                  0c012d60    000002e0                      : _printfi.obj (.text:_pproc_fwp)
                  0c013040    000002a0                      : _printfi.obj (.text:fcvt)
                  0c0132e0    00000280                      : divf.obj (.text:__c6xabi_divf)
                  0c013560    00000280                      : _printfi.obj (.text:ecvt)
                  0c0137e0    00000280                      : memory.obj (.text:free)
                  0c013a60    00000260     Robust_SL2_XMC_MP.obj (.text)
                  0c013cc0    00000240     Robust_DDR_XMC_MP.obj (.text)
                  0c013f00    00000240     Robust_EDMA.obj (.text)
                  0c014140    00000240     Robust_L1_MP.obj (.text)
                  0c014380    00000240     rts6600e_elf.lib : imath64.obj (.text:__c6xabi_divull)
                  0c0145c0    00000240                      : _printfi.obj (.text:_pconv_e)
                  0c014800    00000240                      : _printfi.obj (.text:_pproc_diouxp)
                  0c014a40    00000220     Robust_L1P_ED.obj (.text)
                  0c014c60    00000220     rts6600e_elf.lib : _printfi.obj (.text:_pproc_str)
                  0c014e80    00000220                      : fputc.obj (.text:fputc)
                  0c0150a0    00000200     Robust_Peripherals_MPU.obj (.text)
                  0c0152a0    00000200     Robust_Reserved_space.obj (.text)
                  0c0154a0    00000200     rts6600e_elf.lib : _printfi.obj (.text:_pconv_g)
                  0c0156a0    00000200                      : setvbuf.obj (.text:setvbuf)
                  0c0158a0    000001c0                      : _printfi.obj (.text:_mcpy)
                  0c015a60    000001a0                      : trgdrv.obj (.text:HOSTrename)
                  0c015c00    000001a0     Robust_watch_dog.obj (.text)
                  0c015da0    000001a0     rts6600e_elf.lib : imath40.obj (.text:__c6xabi_divul)
                  0c015f40    00000180                      : copy_decompress_rle.obj (.text:__TI_decompress_rle_core)
                  0c0160c0    00000180                      : memory.obj (.text:malloc)
                  0c016240    00000160     Robust_MNav_Init.obj (.text)
                  0c0163a0    00000140     rts6600e_elf.lib : _printfi.obj (.text:_pproc_fflags)
                  0c0164e0    00000140                      : lowlev.obj (.text:getdevice)
                  0c016620    00000120                      : fclose.obj (.text:_closefile)
                  0c016740    00000120                      : _printfi.obj (.text:_ltostr)
                  0c016860    00000120                      : fseek.obj (.text:fseek)
                  0c016980    00000100                      : trgdrv.obj (.text:HOSTlseek)
                  0c016a80    00000100                      : autoinit.obj (.text:_auto_init_elf)
                  0c016b80    00000100                      : _io_perm.obj (.text:_wrt_ok)
                  0c016c80    00000100                      : cpy_tbl.obj (.text:copy_in)
                  0c016d80    000000e0                      : trgdrv.obj (.text:HOSTopen)
                  0c016e60    000000e0                      : _printfi.obj (.text:_div)
                  0c016f40    000000e0                      : atoi.obj (.text:atoi)
                  0c017020    000000e0                      : lowlev.obj (.text:close)
                  0c017100    000000e0                      : copy_zero_init.obj (.text:decompress:ZI:__TI_zero_init)
                  0c0171e0    000000e0                      : ltoa.obj (.text:ltoa)
                  0c0172c0    000000e0                      : memset.obj (.text:memset)
                  0c0173a0    000000e0                      : printf.obj (.text:printf)
                  0c017480    000000c0                      : trgdrv.obj (.text:HOSTread)
                  0c017540    000000c0                      : trgdrv.obj (.text:HOSTunlink)
                  0c017600    000000c0                      : trgdrv.obj (.text:HOSTwrite)
                  0c0176c0    000000c0                      : divu.obj (.text:__divu)
                  0c017780    000000c0                      : fflush.obj (.text:_doflush)
                  0c017840    000000c0                      : exit.obj (.text:exit)
                  0c017900    000000c0                      : tls.obj (.text:tls:init:__TI_tls_init)
                  0c0179c0    000000a0                      : trgdrv.obj (.text:HOSTclose)
                  0c017a60    000000a0                      : fopen.obj (.text:_cleanup)
                  0c017b00    000000a0                      : _printfi.obj (.text:_ecpy)
                  0c017ba0    000000a0                      : _printfi.obj (.text:_fcpy)
                  0c017c40    000000a0                      : memory.obj (.text:_minit)
                  0c017ce0    000000a0                      : _printfi.obj (.text:_pconv_f)
                  0c017d80    000000a0                      : lowlev.obj (.text:finddevice)
                  0c017e20    000000a0                      : lowlev.obj (.text:lseek)
                  0c017ec0    000000a0                      : memcpy64.obj (.text:memcpy)
                  0c017f60    000000a0                      : memory.obj (.text:minsert)
                  0c018000    000000a0                      : memory.obj (.text:mremove)
                  0c0180a0    000000a0                      : lowlev.obj (.text:write)
                  0c018140    00000080                      : fixdu.obj (.text:__c6xabi_fixdu)
                  0c0181c0    00000080                      : fixfu.obj (.text:__c6xabi_fixfu)
                  0c018240    00000080                      : llshift.obj (.text:__c6xabi_llshl)
                  0c0182c0    00000080                      : boot.obj (.text:_c_int00)
                  0c018340    00000080                      : trgmsg.obj (.text:readmsg)
                  0c0183c0    00000080                      : lowlev.obj (.text:unlink)
                  0c018440    00000060                      : cpp_init.obj (.text:__TI_cpp_init)
                  0c0184a0    00000060                      : frcmpyd_div.obj (.text:__c6xabi_frcmpyd_div)
                  0c018500    00000060                      : llshift.obj (.text:__c6xabi_llshru)
                  0c018560    00000060                      : imath64.obj (.text:_subcull)
                  0c0185c0    00000060                      : memccpy.obj (.text:memccpy)
                  0c018620    00000060                      : trgmsg.obj (.text:writemsg)
                  0c018680    00000040     Robust_vectors.obj (.text)
                  0c0186c0    00000040     rts6600e_elf.lib : isinf.obj (.text:__c6xabi_isinf)
                  0c018700    00000040                      : _printfi.obj (.text:__c6xabi_isnan)
                  0c018740    00000040                      : strasg.obj (.text:__strasgi_64plus)
                  0c018780    00000040                      : args_main.obj (.text:_args_main)
                  0c0187c0    00000040                      : fputs.obj (.text:puts)
                  0c018800    00000020                      : negll.obj (.text:__c6xabi_negll)
                  0c018820    00000020                      : _lock.obj (.text:_nop)
                  0c018840    00000020                      : printf.obj (.text:_outc)
                  0c018860    00000020                      : printf.obj (.text:_outs)
                  0c018880    00000020                      : exit.obj (.text:abort)
                  0c0188a0    00000020                      : copy_decompress_none.obj (.text:decompress:none:__TI_decompress_none)
                  0c0188c0    00000020                      : copy_decompress_rle.obj (.text:decompress:rle24:__TI_decompress_rle24)
                  0c0188e0    00000010     Robust_L1P_ED.obj ($Tramp$S$$funcTest5)
                  0c0188f0    00000010     Robust_LL2_EDC.obj ($Tramp$S$$funcTest1)
                  0c018900    00000010     KeyStone_common.obj ($Tramp$S$$KeyStone_XMC_MPAX_setup)
                  0c018910    00000010     KeyStone_common.obj ($Tramp$S$$KeyStone_MPAX_seg_setup)
                  0c018920    00000010     KeyStone_common.obj ($Tramp$S$$lock_mem_prot_regs)
                  0c018930    00000010     KeyStone_common.obj ($Tramp$S$$unlock_mem_prot_regs)

Sl2EDCCode 
*          0    0c018940    000000c0     
                  0c018940    000000c0     Robust_SL2_EDC.obj (Sl2EDCCode)

msmcSmsMPData_w 
*          0    0c080000    00010000     UNINITIALIZED
                  0c080000    00010000     Robust_SL2_SMS_MP.obj (msmcSmsMPData_w)

sl2MPData_w 
*          0    0c090000    00010000     UNINITIALIZED
                  0c090000    00010000     Robust_SL2_XMC_MP.obj (sl2MPData_w)

PacketData.buffer_SL2 
*          0    0c0a0000    00007800     UNINITIALIZED
                  0c0a0000    00007800     Robust_MNav_Init.obj (PacketData.buffer_SL2)

msmcSmsMPData_r 
*          0    0c0a8000    00004000     UNINITIALIZED
                  0c0a8000    00004000     Robust_SL2_SMS_MP.obj (msmcSmsMPData_r)

sl2MPData_r 
*          0    0c0ac000    00004000     UNINITIALIZED
                  0c0ac000    00004000     Robust_SL2_XMC_MP.obj (sl2MPData_r)

.const     0    0c0b0000    00003480     
                  0c0b0000    00001a34     KeyStone_common.obj (.const:.string)
                  0c0b1a34    00000388     Robust_LL2_EDC.obj (.const:.string)
                  0c0b1dbc    000002b8     Robust_Reserved_space.obj (.const:.string)
                  0c0b2074    000001f8     Robust_DDR_SES_MP.obj (.const:.string)
                  0c0b226c    000001f8     Robust_SL2_SMS_MP.obj (.const:.string)
                  0c0b2464    000001a4     Robust_L1_MP.obj (.const:.string)
                  0c0b2608    0000018c     Robust_Peripherals_MPU.obj (.const:.string)
                  0c0b2794    00000160     Robust_SL2_XMC_MP.obj (.const:.string)
                  0c0b28f4    00000154     KeyStone_Navigator_init_drv.obj (.const:.string)
                  0c0b2a48    00000154     Robust_SL2_EDC.obj (.const:.string)
                  0c0b2b9c    0000011c     Robust_LL2_MP.obj (.const:.string)
                  0c0b2cb8    00000114     Robust_INTC.obj (.const:.string)
                  0c0b2dcc    00000108     Robust_DDR_XMC_MP.obj (.const:.string)
                  0c0b2ed4    00000002     rts6600e_elf.lib : fputs.obj (.const:.string)
                  0c0b2ed6    00000002     --HOLE-- [fill = 0]
                  0c0b2ed8    00000101                      : ctype.obj (.const:.string:_ctypes_)
                  0c0b2fd9    00000003     --HOLE-- [fill = 0]
                  0c0b2fdc    000000f8     Robust_L1P_ED.obj (.const:.string)
                  0c0b30d4    000000ec     Robust_EDMA.obj (.const:.string)
                  0c0b31c0    000000d8     Robust_watch_dog.obj (.const:.string)
                  0c0b3298    000000d4     Robust_SRIO_Init.obj (.const:.string)
                  0c0b336c    0000005c     KeyStone_DDR_Init.obj (.const:.string)
                  0c0b33c8    00000038     KeyStone_common.obj (.const:$P$T0$1)
                  0c0b3400    00000024     KeyStone_SRIO_Init_drv.obj (.const:.string)
                  0c0b3424    00000024     Robust_System.obj (.const:.string)
                  0c0b3448    00000023     rts6600e_elf.lib : _printfi.obj (.const:.string)
                  0c0b346b    00000005     --HOLE-- [fill = 0]
                  0c0b3470    00000010     KeyStone_SRIO_Init_drv.obj (.const:$P$T0$1)

QMSS_Data.Descriptor_SL2 
*          0    0c0b3480    00002880     UNINITIALIZED
                  0c0b3480    00002880     Robust_MNav_Init.obj (QMSS_Data.Descriptor_SL2)

Sl2EDCData 
*          0    0c0b6000    00001000     UNINITIALIZED
                  0c0b6000    00001000     Robust_SL2_EDC.obj (Sl2EDCData)

.cinit     0    0c0b7000    0000085c     
                  0c0b7000    000003aa     (.cinit..fardata.load) [load image, compression = rle]
                  0c0b73aa    00000002     --HOLE-- [fill = 0]
                  0c0b73ac    00000295     (.cinit..far.load) [load image, compression = rle]
                  0c0b7641    00000003     --HOLE-- [fill = 0]
                  0c0b7644    000000f1     (.cinit..neardata.load) [load image, compression = rle]
                  0c0b7735    00000003     --HOLE-- [fill = 0]
                  0c0b7738    00000026     (.cinit.ll2EDCData.load) [load image, compression = rle]
                  0c0b775e    00000002     --HOLE-- [fill = 0]
                  0c0b7760    0000000c     (__TI_handler_table)
                  0c0b776c    00000008     (.cinit..bss.load) [load image, compression = zero_init]
                  0c0b7774    00000008     (.cinit.PacketData.buffer_SL2.load) [load image, compression = zero_init]
                  0c0b777c    00000008     (.cinit.QMSS_Data.Descriptor_SL2.load) [load image, compression = zero_init]
                  0c0b7784    00000008     (.cinit.Sl2EDCData.load) [load image, compression = zero_init]
                  0c0b778c    00000008     (.cinit.ddr3MPData_r.load) [load image, compression = zero_init]
                  0c0b7794    00000008     (.cinit.ddr3MPData_w.load) [load image, compression = zero_init]
                  0c0b779c    00000008     (.cinit.ll2MPData.load) [load image, compression = zero_init]
                  0c0b77a4    00000008     (.cinit.msmcSesMPData_r.load) [load image, compression = zero_init]
                  0c0b77ac    00000008     (.cinit.msmcSesMPData_w.load) [load image, compression = zero_init]
                  0c0b77b4    00000008     (.cinit.msmcSmsMPData_r.load) [load image, compression = zero_init]
                  0c0b77bc    00000008     (.cinit.msmcSmsMPData_w.load) [load image, compression = zero_init]
                  0c0b77c4    00000008     (.cinit.sl2MPData_r.load) [load image, compression = zero_init]
                  0c0b77cc    00000008     (.cinit.sl2MPData_w.load) [load image, compression = zero_init]
                  0c0b77d4    00000088     (__TI_cinit_table)

ddr3MPData_w 
*          0    81000000    00010000     UNINITIALIZED
                  81000000    00010000     Robust_DDR_XMC_MP.obj (ddr3MPData_w)

msmcSesMPData_w 
*          0    81010000    00010000     UNINITIALIZED
                  81010000    00010000     Robust_DDR_SES_MP.obj (msmcSesMPData_w)

ddr3MPData_r 
*          0    81020000    00004000     UNINITIALIZED
                  81020000    00004000     Robust_DDR_XMC_MP.obj (ddr3MPData_r)

msmcSesMPData_r 
*          0    81024000    00004000     UNINITIALIZED
                  81024000    00004000     Robust_DDR_SES_MP.obj (msmcSesMPData_r)


LINKER GENERATED COPY TABLES

__TI_cinit_table @ 0c0b77d4 records: 17, size/record: 8, table size: 136
	.fardata: load addr=0c0b7000, load size=000003aa bytes, run addr=008399a0, run size=000006d4 bytes, compression=rle
	.far: load addr=0c0b73ac, load size=00000295 bytes, run addr=00839000, run size=000009a0 bytes, compression=rle
	.neardata: load addr=0c0b7644, load size=000000f1 bytes, run addr=0083a194, run size=000000f4 bytes, compression=rle
	ll2EDCData: load addr=0c0b7738, load size=00000026 bytes, run addr=0083a2c0, run size=000000a0 bytes, compression=rle
	.bss: load addr=0c0b776c, load size=00000008 bytes, run addr=0083a288, run size=00000014 bytes, compression=zero_init
	PacketData.buffer_SL2: load addr=0c0b7774, load size=00000008 bytes, run addr=0c0a0000, run size=00007800 bytes, compression=zero_init
	QMSS_Data.Descriptor_SL2: load addr=0c0b777c, load size=00000008 bytes, run addr=0c0b3480, run size=00002880 bytes, compression=zero_init
	Sl2EDCData: load addr=0c0b7784, load size=00000008 bytes, run addr=0c0b6000, run size=00001000 bytes, compression=zero_init
	ddr3MPData_r: load addr=0c0b778c, load size=00000008 bytes, run addr=81020000, run size=00004000 bytes, compression=zero_init
	ddr3MPData_w: load addr=0c0b7794, load size=00000008 bytes, run addr=81000000, run size=00010000 bytes, compression=zero_init
	ll2MPData: load addr=0c0b779c, load size=00000008 bytes, run addr=00820000, run size=00010000 bytes, compression=zero_init
	msmcSesMPData_r: load addr=0c0b77a4, load size=00000008 bytes, run addr=81024000, run size=00004000 bytes, compression=zero_init
	msmcSesMPData_w: load addr=0c0b77ac, load size=00000008 bytes, run addr=81010000, run size=00010000 bytes, compression=zero_init
	msmcSmsMPData_r: load addr=0c0b77b4, load size=00000008 bytes, run addr=0c0a8000, run size=00004000 bytes, compression=zero_init
	msmcSmsMPData_w: load addr=0c0b77bc, load size=00000008 bytes, run addr=0c080000, run size=00010000 bytes, compression=zero_init
	sl2MPData_r: load addr=0c0b77c4, load size=00000008 bytes, run addr=0c0ac000, run size=00004000 bytes, compression=zero_init
	sl2MPData_w: load addr=0c0b77cc, load size=00000008 bytes, run addr=0c090000, run size=00010000 bytes, compression=zero_init


LINKER GENERATED HANDLER TABLE

__TI_handler_table @ 0c0b7760 records: 3, size/record: 4, table size: 12
	index: 0, handler: __TI_decompress_rle24
	index: 1, handler: __TI_decompress_none
	index: 2, handler: __TI_zero_init


FAR CALL TRAMPOLINES

callee name               trampoline name
   callee addr  tramp addr   call addr  call info
--------------  -----------  ---------  ----------------
$ll2EDCCode:Robust_L1P_ED.obj$0x0  $Tramp$S$$funcTest5
   00800780     0c0188e0     0c014b6c   Robust_L1P_ED.obj (.text)
                             0c014b90   Robust_L1P_ED.obj (.text)
                             0c014bb4   Robust_L1P_ED.obj (.text)
$ll2EDCCode:Robust_LL2_EDC.obj$0x0  $Tramp$S$$funcTest1
   00800680     0c0188f0     0c00e8d4   Robust_LL2_EDC.obj (.text)
                             0c00e8f8   Robust_LL2_EDC.obj (.text)
$.text:Core_MPAX:KeyStone_common.obj$0x334  $Tramp$S$$KeyStone_XMC_MPAX_setup
   00800534     0c018900     0c00606c   KeyStone_DDR_Init.obj (.text)
                             0c010960   Robust_System.obj (.text)
                             0c0109ac   Robust_System.obj (.text)
                             0c0109ec   Robust_System.obj (.text)
                             0c010a04   Robust_System.obj (.text)
                             0c013b90   Robust_SL2_XMC_MP.obj (.text)
                             0c013e04   Robust_DDR_XMC_MP.obj (.text)
$.text:Core_MPAX:KeyStone_common.obj$0x190  $Tramp$S$$KeyStone_MPAX_seg_setup
   00800390     0c018910     0c002b70   KeyStone_common.obj (.text)
                             0c002c50   KeyStone_common.obj (.text)
                             0c00f7bc   Robust_SL2_EDC.obj (.text)
$.text:Core_MPAX:KeyStone_common.obj$0x0  $Tramp$S$$lock_mem_prot_regs
   00800200     0c018920     0c002650   KeyStone_common.obj (.text)
                             0c0026e4   KeyStone_common.obj (.text)
                             0c002774   KeyStone_common.obj (.text)
                             0c002824   KeyStone_common.obj (.text)
                             0c0029b4   KeyStone_common.obj (.text)
                             0c00f7c8   Robust_SL2_EDC.obj (.text)
$.text:Core_MPAX:KeyStone_common.obj$0xc8  $Tramp$S$$unlock_mem_prot_regs
   008002c8     0c018930     0c0025e4   KeyStone_common.obj (.text)
                             0c002688   KeyStone_common.obj (.text)
                             0c002718   KeyStone_common.obj (.text)
                             0c0027c0   KeyStone_common.obj (.text)
                             0c002860   KeyStone_common.obj (.text)
                             0c00f794   Robust_SL2_EDC.obj (.text)
$.text:KeyStone_common.obj$0x874  $Tramp$S$$CSL_XMC_invalidatePrefetchBuffer
   0c000874     00800640     00800590   KeyStone_common.obj (.text:Core_MPAX)
$.text:KeyStone_common.obj$0x840  $Tramp$S$$CACHE_wbInvAllL2
   0c000840     00800650     00800588   KeyStone_common.obj (.text:Core_MPAX)
$.text:printf:rts6600e_elf.lib<printf.obj>$0x0  $Tramp$S$$printf
   0c0173a0     00800660     008003c8   KeyStone_common.obj (.text:Core_MPAX)
                             008003e0   KeyStone_common.obj (.text:Core_MPAX)
                             00800424   KeyStone_common.obj (.text:Core_MPAX)
                             00800460   KeyStone_common.obj (.text:Core_MPAX)
                             00800488   KeyStone_common.obj (.text:Core_MPAX)
                             008004ac   KeyStone_common.obj (.text:Core_MPAX)
                             008004d4   KeyStone_common.obj (.text:Core_MPAX)
                             00800500   KeyStone_common.obj (.text:Core_MPAX)
                             00800558   KeyStone_common.obj (.text:Core_MPAX)

[9 trampolines]
[38 trampoline calls]


GLOBAL SYMBOLS: SORTED ALPHABETICALLY BY Name 

address    name
--------   ----
0c004770   Bus_error_handler
0c018880   C$$EXIT
0c018678   C$$IO$$
0c007a60   C6657_EVM_DDR_Init
0c0073ec   C6670_EVM_DDR_Init
0c006530   C6678_EVM_DDR_Init
0c013cc0   DDR3MemoryBufInit
0c00600c   DDR3_registers_adress_map
00839938   DDR_MPAX_cfg_table
00839978   DDR_REGS_MPAX_cfg_table
0c006bc8   Dual_Nyquist_EVM_DDR_Init
0c0b6000   EDCTestData
0c0021d4   EDMA_CC_error_handler
0c013f00   EDMA_ERROR_test
0c0023e8   EDMA_TC_error_handler
0c00181c   EDMA_TC_priority_cfg
0c0017b8   EDMA_channel_TC_cfg
0c001b88   EDMA_copy
0c002514   EDMA_error_handler
0c001d94   EDMA_fill
0c001870   EDMA_init
0c001ac8   EDMA_wait
0c005298   EXC_NMI
0c0051d8   EXC_internal
0c0052b0   EXC_swgen
0c00f9a0   Exception_service_routine
0c002f4c   Gauss_MPU4_constant
0c0179c0   HOSTclose
0c016980   HOSTlseek
0c016d80   HOSTopen
0c017480   HOSTread
0c015a60   HOSTrename
0c017540   HOSTunlink
0c017600   HOSTwrite
0c002134   IDMA_copy
0c002108   IDMA_wait
0c0122e0   INT_drop_test
0c010284   InitLsuTransfer
0c00484c   KeyStone_CIC_EXC_handler
0c00406c   KeyStone_CIC_exception_events_mapping
0c00bcb4   KeyStone_Copy_FDQ
0c0029c4   KeyStone_CorePac_AID_map
0c006214   KeyStone_DDR_ECC_INT_enable
0c006238   KeyStone_DDR_ECC_init
0c001130   KeyStone_DDR_PLL_init
0c006424   KeyStone_DDR_clock_phase_init
0c006080   KeyStone_DDR_full_leveling
0c008768   KeyStone_DDR_init
0c0064e4   KeyStone_DDR_latch_leveling_configuration
0c006110   KeyStone_DDR_read_incremental_leveling
0c004d18   KeyStone_EXC_external
0c004564   KeyStone_Exception_cfg
0c00b8a4   KeyStone_Host_Descriptor_Queues_init
0c00d160   KeyStone_HyperLink_Serdes_init
00800390   KeyStone_MPAX_seg_setup
0c003220   KeyStone_MPU_MPPA_modify
0c003324   KeyStone_MPU_interrupts_enable
0c002f8c   KeyStone_MPU_range_setup
0c00300c   KeyStone_MPU_setup
0c002c88   KeyStone_MSMC_MP_interrupt_en
0c002e08   KeyStone_MSMC_protection_exception_handler
0c00bb20   KeyStone_Mono_Descriptor_Queues_init
0c000f98   KeyStone_PLL_init
0c002a4c   KeyStone_PrivID_Remap
0c00b4b8   KeyStone_QMSS_Descriptor_Regions_init
0c00b3e8   KeyStone_QMSS_Linking_RAM_init
0c00bf40   KeyStone_Qmss_Config_Acc_Channel
0c00c270   KeyStone_Qmss_Config_Reclaim_Queue
0c00bd80   KeyStone_Qmss_Download_Firmware
0c00c204   KeyStone_Qmss_config_Acc_Timer
0c00c138   KeyStone_Qmss_disable_Acc_Channel
0c002ba8   KeyStone_SES_MPAX_setup
0c003754   KeyStone_SL2_EDC_enable
0c003d88   KeyStone_SL2_EDC_handler
0c003814   KeyStone_SL2_EDC_interrupt_en
0c002ac8   KeyStone_SMS_MPAX_setup
0c00afe8   KeyStone_SRIO_Build_Type11_Msg_Desc
0c00b130   KeyStone_SRIO_Build_Type9_Msg_Desc
0c009114   KeyStone_SRIO_CSR_CAR_Config
0c009b24   KeyStone_SRIO_Datastreaming_init
0c00ac10   KeyStone_SRIO_DirectIO
0c00ad6c   KeyStone_SRIO_DoorBell
0c009454   KeyStone_SRIO_Error_Capture_Enable
0c00a298   KeyStone_SRIO_Flow_Control
0c009ce4   KeyStone_SRIO_Garbage_Queue_Cfg
0c008ac0   KeyStone_SRIO_GlobalEnable
0c00a3cc   KeyStone_SRIO_Init
0c009fa0   KeyStone_SRIO_Interrupt_init
0c00a884   KeyStone_SRIO_LSU_transfer
0c00acb8   KeyStone_SRIO_Maintenance
0c009e4c   KeyStone_SRIO_MulticastID_Cfg
0c00a230   KeyStone_SRIO_Prioirity_Permission_Setup
0c009ed4   KeyStone_SRIO_RxMode_Setup
0c00cec4   KeyStone_SRIO_Serdes_init
0c009bb0   KeyStone_SRIO_TX_Queue_Cfg
0c008ebc   KeyStone_SRIO_Timeout_Config
0c008c8c   KeyStone_SRIO_disable_all_blocks
0c008b0c   KeyStone_SRIO_enable_blocks
0c00abb0   KeyStone_SRIO_get_LSU_completion_context_code
0c009f90   KeyStone_SRIO_little_endian_swap
0c00ae04   KeyStone_SRIO_match_ACK_ID
0c009d54   KeyStone_SRIO_packet_forwarding_Cfg
0c008e70   KeyStone_SRIO_set_1x2x4x_Path
0c0096a0   KeyStone_SRIO_set_device_ID
0c008d24   KeyStone_SRIO_soft_reset
0c00ab2c   KeyStone_SRIO_wait_LSU_completion
0c00ccc8   KeyStone_Serdes_PLL_config
0c00d620   KeyStone_Serdes_disable
00800534   KeyStone_XMC_MPAX_setup
0c00176c   KeyStone_disable_PSC_Power_Domain
0c001714   KeyStone_disable_PSC_module
0c0016b0   KeyStone_enable_PSC_module
0c000b0c   KeyStone_main_PLL_init
0c0097d4   KeyStone_map_SRIO_RX_message
0c00366c   KeyStone_peripherals_MPU_excepiton_handler
0c00356c   KeyStone_peripherals_MPU_fault_status
0c00c2d8   KeyStone_pktDma_Global_Control
0c00c340   KeyStone_pktDma_TxCh_config
0c00c398   KeyStone_pktDma_configureRxFlow
0c0052c8   KeyStone_print_device_info
0c00d408   Keystone_SGMII_Serdes_init
0c014238   L1D_MP_test
0c0026f0   L1D_memory_protection_cfg
0c014b2c   L1P_Cache_1bit_ERR
0c0039d0   L1P_EDC_setup
0c003c64   L1P_ED_handler
0c014c24   L1P_ED_test
0c014140   L1P_MP_test
0c002660   L1P_memory_protection_cfg
0c0025b8   L1_MPPA_setup
0c002784   L1_cache_protection
0c012720   LL2MemoryBufInit
0083a218   LL2_EDC_DMA_err_str
0c00ee98   LL2_EDC_ISR
0083a21c   LL2_EDC_L1D_err_str
0083a220   LL2_EDC_L1P_err_str
0c003a54   LL2_EDC_handler
0c003934   LL2_EDC_scrub
0c00e7f8   LL2_EDC_scrubbing_timer_setup
0c00386c   LL2_EDC_setup
0c00eca4   LL2_EDC_test
0083a2c0   LL2_EDC_test_Data
0083a300   LL2_EDC_test_Data2
0083a214   LL2_EDC_victim_err_str
0c002794   LL2_MPPA_setup
0c0127b4   LL2_MP_test
0c002830   LL2_Memory_Protection_cfg
0c00e870   LL2_RAM_code_bit_ERR_test
0c00eb08   LL2_RAM_data_bit_ERR_test_byDmaAcess
0c00e908   LL2_RAM_data_bit_ERR_test_byL1dAcess
00839e08   LSU_state_index_table
00839e90   MPU1_cfg_table
00839c20   MPU2_cfg_table
0c00d74c   MSMCSesMemoryBufInit
0c00df0c   MSMCSmsMemoryBufInit
0c005a0c   Memory_Address_Bus_Test
0c005360   Memory_Address_Test
0c0055e0   Memory_Data_Bus_Test
0c0054a4   Memory_Fill_Test
0c005e70   Memory_quick_test
0c00fd50   Nested_Exception_service_routine
0083a040   Ns_str
00839fc0   Peri_MPU_err_type_str
0c01630c   PktDMA_init
0c016280   QMSS_init
0c0150ec   Queue_MP_test
0c01536c   Reserved_Space_Test
0c00136c   Reset_Timer
0c0120f0   Robust_Interrupts_Init
0c00d818   SES_DDR_MP_test
00839f20   SES_MPAX_cfg_table
0c013a60   SL2MemoryBufInit
0c00f0b0   SL2_EDC_ISR
0c00f744   SL2_EDC_test
00839958   SL2_MPAX_cfg_table
0c00f7f8   SL2_code_bit_ERR_test
0c00f8e0   SL2_data_bit_ERR_test
00839f40   SMS_MPAX_cfg_table
0c00dfe0   SMS_SL2_MP_test
0c0103b0   SRIO_Init
0c00166c   Service_Watchdog
0c008098   TCI6614_EVM_DDR_Init
0c002f00   TN_MPU5_constant
0c001228   TSC_delay_ms
0c0012c8   TSC_delay_us
0c001214   TSC_init
0c0013c0   Timer64_Init
0c00ece0   Timer_ISR
0c013da0   XMC_DDR_MP_test
00839400   XMC_MPAX_cfg_table
00839610   XMC_MPAX_cfg_table_C6657
00839560   XMC_MPAX_cfg_table_C6678
008394a0   XMC_MPAX_cfg_table_TCI6614
0c013b40   XMC_SL2_MP_test
0083a074   __CIOBUF_
0c0b77d4   __TI_CINIT_Base
0c0b785c   __TI_CINIT_Limit
0c0b7760   __TI_Handler_Table_Base
0c0b776c   __TI_Handler_Table_Limit
UNDEFED    __TI_INITARRAY_Base
UNDEFED    __TI_INITARRAY_Limit
00839000   __TI_STACK_END
00001000   __TI_STACK_SIZE
0083a194   __TI_STATIC_BASE
00008000   __TI_SYSMEM_SIZE
UNDEFED    __TI_TLS_INIT_Base
UNDEFED    __TI_TLS_INIT_Limit
00000001   __TI_args_main
0c018440   __TI_cpp_init
0c0188a0   __TI_decompress_none
0c0188c0   __TI_decompress_rle24
0083a030   __TI_enable_exit_profile_output
ffffffff   __TI_pprof_out_hndl
ffffffff   __TI_prof_data_size
ffffffff   __TI_prof_data_start
0c017900   __TI_tls_init
0c017100   __TI_zero_init
ffffffff   __binit__
0c010b40   __c6xabi_divd
0c0132e0   __c6xabi_divf
0c0176c0   __c6xabi_divu
0c015da0   __c6xabi_divul
0c014380   __c6xabi_divull
0c018140   __c6xabi_fixdu
0c0181c0   __c6xabi_fixfu
0c0184a0   __c6xabi_frcmpyd_div
0c0186c0   __c6xabi_isinf
0c018240   __c6xabi_llshl
0c018500   __c6xabi_llshru
0c018800   __c6xabi_negll
0c018740   __c6xabi_strasgi_64plus
ffffffff   __c_args__
0c0176c0   __divu
0c018740   __strasgi_64plus
0c018780   _args_main
0c016a80   _auto_init_elf
0c0182c0   _c_int00
0c017a60   _cleanup
0083a028   _cleanup_ptr
0c016620   _closefile
0c0b2ed8   _ctypes_
0c017780   _doflush
0083a02c   _dtors_ptr
00839ca4   _ft_end
008399a0   _ftable
0083a060   _lock
0c017c40   _minit
0c018820   _nop
0c0116c0   _printfi
00838000   _stack
0c018560   _subcull
00830000   _sys_memory
008396c0   _tmpnams
0083a064   _unlock
0c016b80   _wrt_ok
0c018880   abort
0c016f40   atoi
ffffffff   binit
00839f60   bus_err_stat_str
0c0011c0   calc_cycle_measure_overhead
0c017020   close
0c016c80   copy_in
0083a20c   cycle_measure_overhead
81000000   ddr3MPDataDst
81020000   ddr3MPDataSrc
00839fd8   descMemRegionsCfg
0083a068   dsp0_device_ID_routing_config
008398cc   exception_record
0c015338   execute_reserved_space
0c017840   exit
00839d98   flowCfgTable
0c014e80   fputc
0c012380   fputs
0c0137e0   free
00839d20   freeHostQueueCfgTable
0083a008   freeMonoQueueCfgTable
0c016860   fseek
00800680   funcTest1
0c018940   funcTest1_SL2
008006c0   funcTest2
0c018980   funcTest2_SL2
00800700   funcTest3
0c0189c0   funcTest3_SL2
00800740   funcTest4
00800780   funcTest5
00839f80   gCIC_EXC_EN_MASK
0083a228   gCIC_EXC_out_num
0083a280   gCIC_out_num
0083a208   gDSP_Core_Speed_Hz
0c01004c   get_path_string
0083a19c   gpBootCfgRegs
0083a198   gpCGEM_regs
0083a1b0   gpCIC0_regs
0083a1b4   gpCIC1_regs
0083a1b8   gpCIC_regs
0083a204   gpDDR_regs
0083a1bc   gpEDMA_CC2_regs
0083a070   gpEDMA_CC_regs
0083a1c0   gpEDMA_TC_2_0_regs
0083a1c4   gpEDMA_TC_2_1_regs
0083a1c8   gpEDMA_TC_2_2_regs
0083a1cc   gpEDMA_TC_2_3_regs
0083a018   gpEDMA_TC_regs
0083a1ac   gpGPIO_regs
0083a1f4   gpMPU0_regs
0083a1f8   gpMPU1_regs
0083a1fc   gpMPU2_regs
0083a200   gpMPU3_regs
00839fa0   gpMPU_regs
0083a1a8   gpMSMC_regs
0083a1a0   gpPLLC_regs
0083a1a4   gpPSC_regs
0083a250   gpQM_DMA_CfgRegs
0083a258   gpQM_DMA_RxChCfgRegs
0083a260   gpQM_DMA_RxFlowCfgRegs
0083a254   gpQM_DMA_TxChCfgRegs
0083a25c   gpQM_DMA_TxChPriority
0083a24c   gpQM_INTD_regs
0083a048   gpQM_PDSP_Cmd
0083a050   gpQM_PDSP_CtrlRegs
0083a058   gpQM_PDSP_IRAM
0083a22c   gpQM_configRegs
0083a230   gpQM_descriptorRegions
0083a238   gpQueueManageProxyRegs
0083a240   gpQueueManageProxyVBUSM
0083a234   gpQueueManageRegs
0083a23c   gpQueueManageVBUSM
0083a244   gpQueueStatusConfigRegs
0083a248   gpQueueThresholdStatus
0083a264   gpSRIO_DMA_CfgRegs
0083a26c   gpSRIO_DMA_RxChCfgRegs
0083a274   gpSRIO_DMA_RxFlowCfgRegs
0083a268   gpSRIO_DMA_TxChCfgRegs
0083a270   gpSRIO_DMA_TxChPriority
0083a27c   gpSRIO_regs
0083a1d0   gpTimer0Regs
0083a1d4   gpTimer1Regs
0083a1d8   gpTimer2Regs
0083a1dc   gpTimer3Regs
0083a1e0   gpTimer4Regs
0083a1e4   gpTimer5Regs
0083a1e8   gpTimer6Regs
0083a1ec   gpTimer7Regs
0083a1f0   gpTimer8Regs
00839ed0   gpTimerRegs
0083a194   gpXMC_regs
00839e50   gstruMpuAddrRange
0083a224   guwIntcCICExcEvtIdx
0c0b3480   hostDescriptor_SL2
00839ef8   internal_exception_str
00820000   ll2MPDataDst
00839000   ll2MPDataSrc
00800200   lock_mem_prot_regs
0083a284   loopback_mode
0c017e20   lseek
0c0171e0   ltoa
0c01080c   main
0c0160c0   malloc
00839988   mem_prot_key
0c0185c0   memccpy
0c017ec0   memcpy
0c002cf0   memory_protection_exception_handler
0c0172c0   memset
0c0b3c80   monoDescriptor_SL2
00839850   msg_cfg
81010000   msmcSesMPDataDst
81024000   msmcSesMPDataSrc
0c080000   msmcSmsMPDataDst
0c0a8000   msmcSmsMPDataSrc
0083a278   numLinkingEntry
0c0a0000   packetBuffer_SL2_Size0
0c0a0800   packetBuffer_SL2_Size1
0c0a1800   packetBuffer_SL2_Size2
0c0a3800   packetBuffer_SL2_Size3
00839ff0   path_str
0c015218   peripheral_MP_test
0c0173a0   printf
0c0187c0   puts
0c0152a0   read_reserved_space
0c018340   readmsg
0c0183c0   remove
00839824   serdesLinkSetup
00839800   serdes_cfg
0c0156a0   setvbuf
0c090000   sl2MPDataDst
0c0ac000   sl2MPDataSrc
0083a298   srioSerdesRegs
00839870   srio_cfg
0c0100f4   srio_identify_used_ports_lanes
0083a340   temp_LL2_test_Data
0083a28c   uiInitialHostFdqNum
0083a290   uiInitialMonoFdqNum
0083a210   uiLL2_scrub_addr
0083a288   uiUsedDescRegionNum
0083a294   uiUsedRxFlowNum
0c0183c0   unlink
008002c8   unlock_mem_prot_regs
00800000   vectors
0c015c00   watch_dog_test
0c0180a0   write
0c0152d8   write_reserved_space
0c018620   writemsg


GLOBAL SYMBOLS: SORTED BY Symbol Address 

address    name
--------   ----
00000001   __TI_args_main
00001000   __TI_STACK_SIZE
00008000   __TI_SYSMEM_SIZE
00800000   vectors
00800200   lock_mem_prot_regs
008002c8   unlock_mem_prot_regs
00800390   KeyStone_MPAX_seg_setup
00800534   KeyStone_XMC_MPAX_setup
00800680   funcTest1
008006c0   funcTest2
00800700   funcTest3
00800740   funcTest4
00800780   funcTest5
00820000   ll2MPDataDst
00830000   _sys_memory
00838000   _stack
00839000   __TI_STACK_END
00839000   ll2MPDataSrc
00839400   XMC_MPAX_cfg_table
008394a0   XMC_MPAX_cfg_table_TCI6614
00839560   XMC_MPAX_cfg_table_C6678
00839610   XMC_MPAX_cfg_table_C6657
008396c0   _tmpnams
00839800   serdes_cfg
00839824   serdesLinkSetup
00839850   msg_cfg
00839870   srio_cfg
008398cc   exception_record
00839938   DDR_MPAX_cfg_table
00839958   SL2_MPAX_cfg_table
00839978   DDR_REGS_MPAX_cfg_table
00839988   mem_prot_key
008399a0   _ftable
00839c20   MPU2_cfg_table
00839ca4   _ft_end
00839d20   freeHostQueueCfgTable
00839d98   flowCfgTable
00839e08   LSU_state_index_table
00839e50   gstruMpuAddrRange
00839e90   MPU1_cfg_table
00839ed0   gpTimerRegs
00839ef8   internal_exception_str
00839f20   SES_MPAX_cfg_table
00839f40   SMS_MPAX_cfg_table
00839f60   bus_err_stat_str
00839f80   gCIC_EXC_EN_MASK
00839fa0   gpMPU_regs
00839fc0   Peri_MPU_err_type_str
00839fd8   descMemRegionsCfg
00839ff0   path_str
0083a008   freeMonoQueueCfgTable
0083a018   gpEDMA_TC_regs
0083a028   _cleanup_ptr
0083a02c   _dtors_ptr
0083a030   __TI_enable_exit_profile_output
0083a040   Ns_str
0083a048   gpQM_PDSP_Cmd
0083a050   gpQM_PDSP_CtrlRegs
0083a058   gpQM_PDSP_IRAM
0083a060   _lock
0083a064   _unlock
0083a068   dsp0_device_ID_routing_config
0083a070   gpEDMA_CC_regs
0083a074   __CIOBUF_
0083a194   __TI_STATIC_BASE
0083a194   gpXMC_regs
0083a198   gpCGEM_regs
0083a19c   gpBootCfgRegs
0083a1a0   gpPLLC_regs
0083a1a4   gpPSC_regs
0083a1a8   gpMSMC_regs
0083a1ac   gpGPIO_regs
0083a1b0   gpCIC0_regs
0083a1b4   gpCIC1_regs
0083a1b8   gpCIC_regs
0083a1bc   gpEDMA_CC2_regs
0083a1c0   gpEDMA_TC_2_0_regs
0083a1c4   gpEDMA_TC_2_1_regs
0083a1c8   gpEDMA_TC_2_2_regs
0083a1cc   gpEDMA_TC_2_3_regs
0083a1d0   gpTimer0Regs
0083a1d4   gpTimer1Regs
0083a1d8   gpTimer2Regs
0083a1dc   gpTimer3Regs
0083a1e0   gpTimer4Regs
0083a1e4   gpTimer5Regs
0083a1e8   gpTimer6Regs
0083a1ec   gpTimer7Regs
0083a1f0   gpTimer8Regs
0083a1f4   gpMPU0_regs
0083a1f8   gpMPU1_regs
0083a1fc   gpMPU2_regs
0083a200   gpMPU3_regs
0083a204   gpDDR_regs
0083a208   gDSP_Core_Speed_Hz
0083a20c   cycle_measure_overhead
0083a210   uiLL2_scrub_addr
0083a214   LL2_EDC_victim_err_str
0083a218   LL2_EDC_DMA_err_str
0083a21c   LL2_EDC_L1D_err_str
0083a220   LL2_EDC_L1P_err_str
0083a224   guwIntcCICExcEvtIdx
0083a228   gCIC_EXC_out_num
0083a22c   gpQM_configRegs
0083a230   gpQM_descriptorRegions
0083a234   gpQueueManageRegs
0083a238   gpQueueManageProxyRegs
0083a23c   gpQueueManageVBUSM
0083a240   gpQueueManageProxyVBUSM
0083a244   gpQueueStatusConfigRegs
0083a248   gpQueueThresholdStatus
0083a24c   gpQM_INTD_regs
0083a250   gpQM_DMA_CfgRegs
0083a254   gpQM_DMA_TxChCfgRegs
0083a258   gpQM_DMA_RxChCfgRegs
0083a25c   gpQM_DMA_TxChPriority
0083a260   gpQM_DMA_RxFlowCfgRegs
0083a264   gpSRIO_DMA_CfgRegs
0083a268   gpSRIO_DMA_TxChCfgRegs
0083a26c   gpSRIO_DMA_RxChCfgRegs
0083a270   gpSRIO_DMA_TxChPriority
0083a274   gpSRIO_DMA_RxFlowCfgRegs
0083a278   numLinkingEntry
0083a27c   gpSRIO_regs
0083a280   gCIC_out_num
0083a284   loopback_mode
0083a288   uiUsedDescRegionNum
0083a28c   uiInitialHostFdqNum
0083a290   uiInitialMonoFdqNum
0083a294   uiUsedRxFlowNum
0083a298   srioSerdesRegs
0083a2c0   LL2_EDC_test_Data
0083a300   LL2_EDC_test_Data2
0083a340   temp_LL2_test_Data
0c000b0c   KeyStone_main_PLL_init
0c000f98   KeyStone_PLL_init
0c001130   KeyStone_DDR_PLL_init
0c0011c0   calc_cycle_measure_overhead
0c001214   TSC_init
0c001228   TSC_delay_ms
0c0012c8   TSC_delay_us
0c00136c   Reset_Timer
0c0013c0   Timer64_Init
0c00166c   Service_Watchdog
0c0016b0   KeyStone_enable_PSC_module
0c001714   KeyStone_disable_PSC_module
0c00176c   KeyStone_disable_PSC_Power_Domain
0c0017b8   EDMA_channel_TC_cfg
0c00181c   EDMA_TC_priority_cfg
0c001870   EDMA_init
0c001ac8   EDMA_wait
0c001b88   EDMA_copy
0c001d94   EDMA_fill
0c002108   IDMA_wait
0c002134   IDMA_copy
0c0021d4   EDMA_CC_error_handler
0c0023e8   EDMA_TC_error_handler
0c002514   EDMA_error_handler
0c0025b8   L1_MPPA_setup
0c002660   L1P_memory_protection_cfg
0c0026f0   L1D_memory_protection_cfg
0c002784   L1_cache_protection
0c002794   LL2_MPPA_setup
0c002830   LL2_Memory_Protection_cfg
0c0029c4   KeyStone_CorePac_AID_map
0c002a4c   KeyStone_PrivID_Remap
0c002ac8   KeyStone_SMS_MPAX_setup
0c002ba8   KeyStone_SES_MPAX_setup
0c002c88   KeyStone_MSMC_MP_interrupt_en
0c002cf0   memory_protection_exception_handler
0c002e08   KeyStone_MSMC_protection_exception_handler
0c002f00   TN_MPU5_constant
0c002f4c   Gauss_MPU4_constant
0c002f8c   KeyStone_MPU_range_setup
0c00300c   KeyStone_MPU_setup
0c003220   KeyStone_MPU_MPPA_modify
0c003324   KeyStone_MPU_interrupts_enable
0c00356c   KeyStone_peripherals_MPU_fault_status
0c00366c   KeyStone_peripherals_MPU_excepiton_handler
0c003754   KeyStone_SL2_EDC_enable
0c003814   KeyStone_SL2_EDC_interrupt_en
0c00386c   LL2_EDC_setup
0c003934   LL2_EDC_scrub
0c0039d0   L1P_EDC_setup
0c003a54   LL2_EDC_handler
0c003c64   L1P_ED_handler
0c003d88   KeyStone_SL2_EDC_handler
0c00406c   KeyStone_CIC_exception_events_mapping
0c004564   KeyStone_Exception_cfg
0c004770   Bus_error_handler
0c00484c   KeyStone_CIC_EXC_handler
0c004d18   KeyStone_EXC_external
0c0051d8   EXC_internal
0c005298   EXC_NMI
0c0052b0   EXC_swgen
0c0052c8   KeyStone_print_device_info
0c005360   Memory_Address_Test
0c0054a4   Memory_Fill_Test
0c0055e0   Memory_Data_Bus_Test
0c005a0c   Memory_Address_Bus_Test
0c005e70   Memory_quick_test
0c00600c   DDR3_registers_adress_map
0c006080   KeyStone_DDR_full_leveling
0c006110   KeyStone_DDR_read_incremental_leveling
0c006214   KeyStone_DDR_ECC_INT_enable
0c006238   KeyStone_DDR_ECC_init
0c006424   KeyStone_DDR_clock_phase_init
0c0064e4   KeyStone_DDR_latch_leveling_configuration
0c006530   C6678_EVM_DDR_Init
0c006bc8   Dual_Nyquist_EVM_DDR_Init
0c0073ec   C6670_EVM_DDR_Init
0c007a60   C6657_EVM_DDR_Init
0c008098   TCI6614_EVM_DDR_Init
0c008768   KeyStone_DDR_init
0c008ac0   KeyStone_SRIO_GlobalEnable
0c008b0c   KeyStone_SRIO_enable_blocks
0c008c8c   KeyStone_SRIO_disable_all_blocks
0c008d24   KeyStone_SRIO_soft_reset
0c008e70   KeyStone_SRIO_set_1x2x4x_Path
0c008ebc   KeyStone_SRIO_Timeout_Config
0c009114   KeyStone_SRIO_CSR_CAR_Config
0c009454   KeyStone_SRIO_Error_Capture_Enable
0c0096a0   KeyStone_SRIO_set_device_ID
0c0097d4   KeyStone_map_SRIO_RX_message
0c009b24   KeyStone_SRIO_Datastreaming_init
0c009bb0   KeyStone_SRIO_TX_Queue_Cfg
0c009ce4   KeyStone_SRIO_Garbage_Queue_Cfg
0c009d54   KeyStone_SRIO_packet_forwarding_Cfg
0c009e4c   KeyStone_SRIO_MulticastID_Cfg
0c009ed4   KeyStone_SRIO_RxMode_Setup
0c009f90   KeyStone_SRIO_little_endian_swap
0c009fa0   KeyStone_SRIO_Interrupt_init
0c00a230   KeyStone_SRIO_Prioirity_Permission_Setup
0c00a298   KeyStone_SRIO_Flow_Control
0c00a3cc   KeyStone_SRIO_Init
0c00a884   KeyStone_SRIO_LSU_transfer
0c00ab2c   KeyStone_SRIO_wait_LSU_completion
0c00abb0   KeyStone_SRIO_get_LSU_completion_context_code
0c00ac10   KeyStone_SRIO_DirectIO
0c00acb8   KeyStone_SRIO_Maintenance
0c00ad6c   KeyStone_SRIO_DoorBell
0c00ae04   KeyStone_SRIO_match_ACK_ID
0c00afe8   KeyStone_SRIO_Build_Type11_Msg_Desc
0c00b130   KeyStone_SRIO_Build_Type9_Msg_Desc
0c00b3e8   KeyStone_QMSS_Linking_RAM_init
0c00b4b8   KeyStone_QMSS_Descriptor_Regions_init
0c00b8a4   KeyStone_Host_Descriptor_Queues_init
0c00bb20   KeyStone_Mono_Descriptor_Queues_init
0c00bcb4   KeyStone_Copy_FDQ
0c00bd80   KeyStone_Qmss_Download_Firmware
0c00bf40   KeyStone_Qmss_Config_Acc_Channel
0c00c138   KeyStone_Qmss_disable_Acc_Channel
0c00c204   KeyStone_Qmss_config_Acc_Timer
0c00c270   KeyStone_Qmss_Config_Reclaim_Queue
0c00c2d8   KeyStone_pktDma_Global_Control
0c00c340   KeyStone_pktDma_TxCh_config
0c00c398   KeyStone_pktDma_configureRxFlow
0c00ccc8   KeyStone_Serdes_PLL_config
0c00cec4   KeyStone_SRIO_Serdes_init
0c00d160   KeyStone_HyperLink_Serdes_init
0c00d408   Keystone_SGMII_Serdes_init
0c00d620   KeyStone_Serdes_disable
0c00d74c   MSMCSesMemoryBufInit
0c00d818   SES_DDR_MP_test
0c00df0c   MSMCSmsMemoryBufInit
0c00dfe0   SMS_SL2_MP_test
0c00e7f8   LL2_EDC_scrubbing_timer_setup
0c00e870   LL2_RAM_code_bit_ERR_test
0c00e908   LL2_RAM_data_bit_ERR_test_byL1dAcess
0c00eb08   LL2_RAM_data_bit_ERR_test_byDmaAcess
0c00eca4   LL2_EDC_test
0c00ece0   Timer_ISR
0c00ee98   LL2_EDC_ISR
0c00f0b0   SL2_EDC_ISR
0c00f744   SL2_EDC_test
0c00f7f8   SL2_code_bit_ERR_test
0c00f8e0   SL2_data_bit_ERR_test
0c00f9a0   Exception_service_routine
0c00fd50   Nested_Exception_service_routine
0c01004c   get_path_string
0c0100f4   srio_identify_used_ports_lanes
0c010284   InitLsuTransfer
0c0103b0   SRIO_Init
0c01080c   main
0c010b40   __c6xabi_divd
0c0116c0   _printfi
0c0120f0   Robust_Interrupts_Init
0c0122e0   INT_drop_test
0c012380   fputs
0c012720   LL2MemoryBufInit
0c0127b4   LL2_MP_test
0c0132e0   __c6xabi_divf
0c0137e0   free
0c013a60   SL2MemoryBufInit
0c013b40   XMC_SL2_MP_test
0c013cc0   DDR3MemoryBufInit
0c013da0   XMC_DDR_MP_test
0c013f00   EDMA_ERROR_test
0c014140   L1P_MP_test
0c014238   L1D_MP_test
0c014380   __c6xabi_divull
0c014b2c   L1P_Cache_1bit_ERR
0c014c24   L1P_ED_test
0c014e80   fputc
0c0150ec   Queue_MP_test
0c015218   peripheral_MP_test
0c0152a0   read_reserved_space
0c0152d8   write_reserved_space
0c015338   execute_reserved_space
0c01536c   Reserved_Space_Test
0c0156a0   setvbuf
0c015a60   HOSTrename
0c015c00   watch_dog_test
0c015da0   __c6xabi_divul
0c0160c0   malloc
0c016280   QMSS_init
0c01630c   PktDMA_init
0c016620   _closefile
0c016860   fseek
0c016980   HOSTlseek
0c016a80   _auto_init_elf
0c016b80   _wrt_ok
0c016c80   copy_in
0c016d80   HOSTopen
0c016f40   atoi
0c017020   close
0c017100   __TI_zero_init
0c0171e0   ltoa
0c0172c0   memset
0c0173a0   printf
0c017480   HOSTread
0c017540   HOSTunlink
0c017600   HOSTwrite
0c0176c0   __c6xabi_divu
0c0176c0   __divu
0c017780   _doflush
0c017840   exit
0c017900   __TI_tls_init
0c0179c0   HOSTclose
0c017a60   _cleanup
0c017c40   _minit
0c017e20   lseek
0c017ec0   memcpy
0c0180a0   write
0c018140   __c6xabi_fixdu
0c0181c0   __c6xabi_fixfu
0c018240   __c6xabi_llshl
0c0182c0   _c_int00
0c018340   readmsg
0c0183c0   remove
0c0183c0   unlink
0c018440   __TI_cpp_init
0c0184a0   __c6xabi_frcmpyd_div
0c018500   __c6xabi_llshru
0c018560   _subcull
0c0185c0   memccpy
0c018620   writemsg
0c018678   C$$IO$$
0c0186c0   __c6xabi_isinf
0c018740   __c6xabi_strasgi_64plus
0c018740   __strasgi_64plus
0c018780   _args_main
0c0187c0   puts
0c018800   __c6xabi_negll
0c018820   _nop
0c018880   C$$EXIT
0c018880   abort
0c0188a0   __TI_decompress_none
0c0188c0   __TI_decompress_rle24
0c018940   funcTest1_SL2
0c018980   funcTest2_SL2
0c0189c0   funcTest3_SL2
0c080000   msmcSmsMPDataDst
0c090000   sl2MPDataDst
0c0a0000   packetBuffer_SL2_Size0
0c0a0800   packetBuffer_SL2_Size1
0c0a1800   packetBuffer_SL2_Size2
0c0a3800   packetBuffer_SL2_Size3
0c0a8000   msmcSmsMPDataSrc
0c0ac000   sl2MPDataSrc
0c0b2ed8   _ctypes_
0c0b3480   hostDescriptor_SL2
0c0b3c80   monoDescriptor_SL2
0c0b6000   EDCTestData
0c0b7760   __TI_Handler_Table_Base
0c0b776c   __TI_Handler_Table_Limit
0c0b77d4   __TI_CINIT_Base
0c0b785c   __TI_CINIT_Limit
81000000   ddr3MPDataDst
81010000   msmcSesMPDataDst
81020000   ddr3MPDataSrc
81024000   msmcSesMPDataSrc
ffffffff   __TI_pprof_out_hndl
ffffffff   __TI_prof_data_size
ffffffff   __TI_prof_data_start
ffffffff   __binit__
ffffffff   __c_args__
ffffffff   binit
UNDEFED    __TI_INITARRAY_Base
UNDEFED    __TI_INITARRAY_Limit
UNDEFED    __TI_TLS_INIT_Base
UNDEFED    __TI_TLS_INIT_Limit

[402 symbols]
